:020000040000FA
:10000000DB28FF3FFF3FFF3F6D28FF3FFF3FFF3FE4
:10001000FF3FA101A201051E0B28051A0D28051E90
:100020000F28A10F1428A20A1528051A1128A10FBC
:100030001A28A20A1B28051E17280230A107031C34
:10004000A20CA10CA20CA10C08000830A4000130E5
:100050002107A200A20C6400051A2B286920051AAA
:100060002528322865200310051A0314A30C00006C
:10007000A40B32286520051EA3012308A000080058
:100080006400A300831603130512831203130830C0
:10009000A400051265204C280000A30C031C562860
:1000A000000005166520A40B4D285B28051265206D
:1000B000A40B4D285B285C280000051665208316DC
:1000C0000313051683120313080004302102A20053
:1000D0000000A20B68286C2808000B188028130861
:1000E0002D0203197E28031C93030318930A130F90
:1000F0007C28051595017E280C3095000B11090010
:10010000051AD92806308F02031C9928B8308E02B0
:10011000031C8F038F1B99280430A5008F0C8E0CB5
:10012000A50B8E280E089F3C03189B289F308E003D
:100130009B2800308E00721ABF28AC0FAF287216B1
:100140002A08831603139A00FC309B00FD202B081D
:10015000831603139A00FB309B00FD20BF28193043
:100160002C02031CBF282A080E020318B9280E0807
:10017000AA000E082B020318BF280E08AB000E08B9
:100180002702031CC828DE30050520388500CC284E
:10019000DE300505013885000E0829020318D22833
:1001A000FF30D528D3280E08F520AD008F018E0131
:1001B000F4200B100900962210100C108F018E01F4
:1001C00010140C181029051AE128AD018F018E01B9
:1001D0003230A600721105080B100B118B17721D1F
:1001E000EF288B139301DC280800831603139B0070
:1001F0001C141A0883120313080083160313F21148
:100200001C1555309D00AA309D009C149C18062991
:100210001A081C141A06031DF21583120313080092
:1002200009200330F30025202008031D1C29F30BAF
:100230001329851D19291029413A03194D29200830
:10024000613A031947292008543A03194A2920081A
:10025000633A0319B3292008433A0319BF29200838
:100260006D3A0319DF2920084D3A0319CB292008DC
:10027000523A0319F3292008563A0319072A20088D
:100280000D3A031D45296222112960221129721796
:10029000F2124E29F21672134E29F2126022252014
:1002A0004422F21C3F29F10120082C226022252043
:1002B0004422F21C3F2920082C22602225202008FD
:1002C0000D3A0319682920083D3A03197F293F296F
:1002D000721B7829F21E72290030F10771089F3CC9
:1002E000031C3F2960227108F5200F226222112988
:1002F00060227108840000080F2262221129F21E78
:1003000087290030F10771089F3C031C3F297108C1
:10031000831603139B0083120313602225204422BB
:10032000F21C3F29F10120082C22602225204422C2
:10033000F21C3F2920082C226022252020080D3A9B
:10034000031D3F297107831603139A00721BAB2903
:10035000FD20622211291B0884001A0880008312E4
:100360000313622211296022252020080D3A031D63
:100370003F296022FC30F5200F22622211296022E1
:10038000252020080D3A031D3F296022FB30F5206F
:100390000F22622211296022252020080D3A031D18
:1003A000D7296022FD30F5200F2262221129200872
:1003B0003D3A0319DC293F29FD30F10087296022ED
:1003C000252020080D3A031DEB296022FE30F52080
:1003D0000F226222112920083D3A0319F0293F29F2
:1003E000FE30F10087296022252020080D3A031DE8
:1003F000FF296022FF30F5200F22622211292008F8
:100400003D3A0319042A3F29FF30F1008729602271
:10041000252020080D3A031D3F2966221129831249
:100420000313AF002F0E0F3922222E08831203135D
:100430004020831203132F080F3922222E08831223
:1004400003134028AE000A302E02031C292A07306D
:10045000AE073030AE07003483120313AE006130B4
:100460002E02031C352A2030AE023A302E02031C25
:100470003B2AF930AE07D030AE070F302E0583127D
:100480000313F10EF104003430302002031C5C2A07
:100490003A302002031C5E2A41302002031C5C2AF1
:1004A00047302002031C5E2A61302002031C5C2AB4
:1004B00067302002031C5E2AF2100034F21400346C
:1004C000200840280D3040203E3040287530F00094
:1004D00002308A0070087422003A03190034402068
:1004E000F00F6A2A8A0A6A2A82000D3430344434B2
:1004F0002C34303432342E34303431342C343034E3
:1005000037343234343432343034303437342C34B9
:10051000313432342C34383446342C344134303491
:100520002C34463446340D343E34003483120313E5
:10053000083085008316031385150516051105106F
:100540008512033081008B1670308F0022309F009F
:10055000FF30920016168B15831203130730990093
:1005600005309F000430920093010C309500C1309B
:100570009000F201FF30F520A700FD30F520A90022
:10058000FE30F520A800FF30AA00AB01AC01080046
:1005900000340034FF3FFF3FFF3FFF3FFF3FFF3F7F
:1005A000FF3FFF3FFF3FFF3FFF3FFF3FFF3FFF3F5B
:1005B000FF3FFF3FFF3FFF3FFF3FFF3FFF3FFF3F4B
:1005C000FF3FFF3FFF3FFF3FFF3FFF3FFF3FFF3F3B
:1005D000FF3FFF3FFF3FFF3FFF3FFF3FFF3FFF3F2B
:104200000000830083008300830083008300830019
:104210008300830083008300830083008300830086
:104220008300830084008400840084008400840070
:10423000840084008400840084008400840084005E
:104240008400840084007D0075006E0066005E00BE
:1042500056004F0047003F00370030002800200084
:10426000180011000900010000000000000000001B
:10427000000000000000000000000000000000003E
:10428000010006000A000F00140018001D002200A3
:1042900026002B003000350039003E004300470067
:1042A0004C00510055005A005F00630068006D002B
:1042B000710076007B007F00840089008E009200F0
:1042C00097009C00A000A500AA00AE00B300B800B3
:1042D000BC00C100C600CA00CF00D400D900DD0078
:1042E000E200E700EB00F000F500F900FF00FF003E
:1042F000FF00FF00FF00FF00FF00FF00FF00FF00C6
:10430000FF00FF00FF00FF00FF00FF00FF00FF00B5
:10431000FF00FF00FF00FF00FF00FF00FF00FF00A5
:10432000FF00FF00FF00FF00FF00FF00FF00FF0095
:10433000FF00FF00FF00FF00FF00FF00FF00FF0085
:10434000FF00FF00FF00FF00FF00FF00FF00FF0075
:10435000FF00FF00FF00FF00FF00FF00FF00FF0065
:10436000FF00FF00FF00FF00FF00FF00FF00FF0055
:10437000FF00FF00FF00FF00FF00FF00FF00FF0045
:10438000FF00FF00FF00FF00FF00FF00FF00FF0035
:10439000FF00FF00FF00FF00FF00FF00FF00FF0025
:1043A000FF00FF00FF00FF00FF00FF00FF00FF0015
:1043B000FF00FF00FF00FF00FF00FF00FF00FF0005
:1043C000FF00FF00FF00FF00FF00FF00FF00FF00F5
:1043D000FF00FF00FF00FF00FF00FF00FF00FF00E5
:1043E000FF00FF00FF00FF00FF00FF00FF00FF00D5
:1043F000FF00FF00FF004B004A0074000A003A0073
:02400E00D433A9
:08400000FF3FFF3FFF3FFF3FC0
:00000001FF
